 flexcansdk

 Timestamp is 4fb04cc1 (Mon May 14 12:07:29 2012)

 Preferred load address is 10000000

 Start         Length     Name                   Class
 0001:00000000 00000004H .CRT$XCA                CODE
 0001:00000004 00000004H .CRT$XCZ                CODE
 0001:00000008 00000004H .CRT$XIA                CODE
 0001:0000000c 00000004H .CRT$XIZ                CODE
 0001:00000010 00000004H .CRT$XPA                CODE
 0001:00000014 00000004H .CRT$XPZ                CODE
 0001:00000018 00000004H .CRT$XTA                CODE
 0001:0000001c 00000004H .CRT$XTZ                CODE
 0001:00000020 0000002aH .rdata                  CODE
 0001:0000004c 00000027H .rdata$debug            CODE
 0001:00000074 00000bf0H .text                   CODE
 0001:00000c64 00000020H .xdata                  CODE
 0001:00000c84 00000014H .idata$2                CODE
 0001:00000c98 00000014H .idata$3                CODE
 0001:00000cac 00000044H .idata$4                CODE
 0001:00000cf0 0000000cH .idata$6                CODE
 0001:00000d00 000000eeH .edata                  CODE
 0002:00000000 00000044H .idata$5                DATA
 0002:00000048 0000044cH .data                   DATA
 0002:00000498 0000001cH .bss                    DATA
 0003:00000000 000000b0H .pdata                  DATA

  Address         Publics by Value              Rva+Base       Lib:Object

 0000:00000000       ___safe_se_handler_count   00000000     <absolute>
 0000:00000000       ___safe_se_handler_table   00000000     <absolute>
 0001:00000000       __xc_a                     10001000     corelib0:crt0init.obj
 0001:00000004       __xc_z                     10001004     corelib0:crt0init.obj
 0001:00000008       __xi_a                     10001008     corelib0:crt0init.obj
 0001:0000000c       __xi_z                     1000100c     corelib0:crt0init.obj
 0001:00000010       __xp_a                     10001010     corelib0:crt0init.obj
 0001:00000014       __xp_z                     10001014     corelib0:crt0init.obj
 0001:00000018       __xt_a                     10001018     corelib0:crt0init.obj
 0001:0000001c       __xt_z                     1000101c     corelib0:crt0init.obj
 0001:0000003c       ??_C@_1O@IFEMKBCF@?$AAC?$AAA?$AAN?$AA?$CF?$AAd?$AA?3?$AA?$AA@ 1000103c     flexcansdk.obj
 0001:00000074       DllMain                    10001074 f   flexcansdk.obj
 0001:00000094       FlexCANInit                10001094 f   flexcansdk.obj
 0001:0000013c       FlexCANDeinit              1000113c f   flexcansdk.obj
 0001:0000042c       FlexCANWriteFrame          1000142c f   flexcansdk.obj
 0001:0000054c       FlexCANReadFrame           1000154c f   flexcansdk.obj
 0001:00000648       FlexCANTransfer            10001648 f   flexcansdk.obj
 0001:000006b4       ??$FlexCANGet@K@@YAHKHPAK@Z 100016b4 f i flexcansdk.obj
 0001:00000714       FlexCANSetBitrate          10001714 f   flexcansdk.obj
 0001:00000780       FlexCANGetBitrate          10001780 f   flexcansdk.obj
 0001:0000079c       DisableThreadLibraryCalls  1000179c f   coredll:COREDLL.dll
 0001:000007ac       CreateFileW                100017ac f   coredll:COREDLL.dll
 0001:000007bc       CloseHandle                100017bc f   coredll:COREDLL.dll
 0001:000007cc       SetLastError               100017cc f   coredll:COREDLL.dll
 0001:000007dc       DeviceIoControl            100017dc f   coredll:COREDLL.dll
 0001:000008f0       _DllMainCRTStartup         100018f0 f   corelib0:pegdmain.obj
 0001:00000920       __GSHandlerCheckCommon     10001920 f   corelib0:gshandler.obj
 0001:0000095c       __GSHandlerCheck           1000195c f   corelib0:gshandler.obj
 0001:00000980       __security_init_cookie     10001980 f   corelib0:seccinit.obj
 0001:000009dc       __security_check_cookie    100019dc f   corelib0:armsecgs.obj
 0001:000009f0       __gsfailure                100019f0 f   corelib0:armsecgs.obj
 0001:00000b30       _cexit                     10001b30 f   corelib0:cexit.obj
 0001:00000b4c       _initterm                  10001b4c f   corelib0:crt0dat.obj
 0001:00000b80       _cinit                     10001b80 f   corelib0:crt0dat.obj
 0001:00000bb4       swprintf                   10001bb4 f   corelib1:COREDLL.dll
 0001:00000bc4       memcpy                     10001bc4 f   corelib1:COREDLL.dll
 0001:00000bd4       memset                     10001bd4 f   corelib1:COREDLL.dll
 0001:00000be4       _XcptFilter                10001be4 f   corelib1:COREDLL.dll
 0001:00000bf4       __C_specific_handler       10001bf4 f   corelib1:COREDLL.dll
 0001:00000c04       __security_gen_cookie2     10001c04 f   corelib1:COREDLL.dll
 0001:00000c14       __report_gsfailure         10001c14 f   corelib1:COREDLL.dll
 0001:00000c24       free                       10001c24 f   corelib1:COREDLL.dll
 0001:00000c34       DeleteCriticalSection      10001c34 f   coredll:COREDLL.dll
 0001:00000c44       InterlockedExchange        10001c44 f   coredll:COREDLL.dll
 0001:00000c54       TerminateProcess           10001c54 f   coredll:COREDLL.dll
 0001:00000c84       __IMPORT_DESCRIPTOR_COREDLL 10001c84     coredll:COREDLL.dll
 0001:00000c98       __NULL_IMPORT_DESCRIPTOR   10001c98     coredll:COREDLL.dll
 0002:00000000       __imp_DisableThreadLibraryCalls 10002000     coredll:COREDLL.dll
 0002:00000004       __imp_CreateFileW          10002004     coredll:COREDLL.dll
 0002:00000008       __imp_CloseHandle          10002008     coredll:COREDLL.dll
 0002:0000000c       __imp_SetLastError         1000200c     coredll:COREDLL.dll
 0002:00000010       __imp_DeviceIoControl      10002010     coredll:COREDLL.dll
 0002:00000014       __imp_swprintf             10002014     corelib1:COREDLL.dll
 0002:00000018       __imp_memcpy               10002018     corelib1:COREDLL.dll
 0002:0000001c       __imp_memset               1000201c     corelib1:COREDLL.dll
 0002:00000020       __imp__XcptFilter          10002020     corelib1:COREDLL.dll
 0002:00000024       __imp___C_specific_handler 10002024     corelib1:COREDLL.dll
 0002:00000028       __imp___security_gen_cookie2 10002028     corelib1:COREDLL.dll
 0002:0000002c       __imp___report_gsfailure   1000202c     corelib1:COREDLL.dll
 0002:00000030       __imp_free                 10002030     corelib1:COREDLL.dll
 0002:00000034       __imp_DeleteCriticalSection 10002034     coredll:COREDLL.dll
 0002:00000038       __imp_InterlockedExchange  10002038     coredll:COREDLL.dll
 0002:0000003c       __imp_TerminateProcess     1000203c     coredll:COREDLL.dll
 0002:00000040       \177COREDLL_NULL_THUNK_DATA 10002040     coredll:COREDLL.dll
 0002:00000048       ?dpCurSettings@@3U_DBGPARAM@@A 10002048     DebugZones.obj
 0002:0000048c       __security_cookie          1000248c     corelib0:seccinit.obj
 0002:00000490       __security_cookie_complement 10002490     corelib0:seccinit.obj
 0002:000004a0       _exitflag                  100024a0     corelib0:cexit.obj
 0002:000004a4       __onexitend                100024a4     <common>
 0002:000004a8       __onexitbegin              100024a8     <common>
 0002:000004ac       g_pcsExit                  100024ac     <common>
 0002:000004b0       _pRawDllMain               100024b0     <common>

 entry point at        0001:000008f0

 Static symbols

 0001:0000018c       ??$CallDriver@UCAN_TRANSFER_BLOCK@@@@YAHKHPAUCAN_TRANSFER_BLOCK@@W4ARGUMENTIO@@@Z 1000118c f   flexcansdk.obj
 0001:000002e0       ??$CallDriver@K@@YAHKHPAKW4ARGUMENTIO@@@Z 100012e0 f   flexcansdk.obj
 0001:000007f4       _DllMainCRTStartupHelper   100017f4 f   corelib0:pegdmain.obj
 0001:00000a34       doexit                     10001a34 f   corelib0:cexit.obj
